:100000000C9466010C948E010C948E010C948E015C
:100010000C948E010C948E010C948E010C948E0124
:100020000C948E010C948E010C9483060C944F0555
:100030000C948E010C948E010C948E010C948E0104
:100040000C948E010C948E010C948E010C948E01F4
:100050000C948E010C948E010C948E010C94A801CA
:100060000C948E010C948E010C948E010C948E01D4
:100070000C948E010C948E010C948E010C948E01C4
:100080000C948E010C948E010C948E010C948E01B4
:100090000C948E010C948E010C948E010C948E01A4
:1000A0000C948E010C948E010C948E01AB02AE0266
:1000B0009D02A102A702CF02CF02CF02B202B60276
:1000C000BA02C002C402CF02CA0200000002000944
:1000D0000F0000030401000C0000000000000000FD
:1000E00000000000000000000408020110408040F1
:1000F000102040804080080204018040201002014E
:10010000108010204040040404040403040502028B
:1001100002020403020202020606060606060404A0
:100120000202020400000000250028002B002E001F
:10013000310000000000240027002A002D003000BC
:1001400000C18081C112010002020000404123373A
:100150008000010102000112010002000000404184
:1001600023378000010102000141726475696E6FDE
:10017000204C4C430041726475696E6F204D696379
:10018000726F0004030904080B0002020201000957
:1001900004000001020200000524001001052401F2
:1001A000010104240206052406000107058103104D
:1001B000004009040100020A000000070502024095
:1001C000000007058302400000000000000000005E
:1001D000002A2B28000000000000000000000000A2
:1001E0000000000000000000002C9EB4A0A1A2A40A
:1001F00034A6A7A5AE362D3738271E1F202122236F
:10020000242526B333B62EB7B89F84858687888980
:100210008A8B8C8D8E8F90919293949596979899C6
:100220009A9B9C9D2F3130A3AD3504050607080924
:100230000A0B0C0D0E0F10111213141516171819A6
:100240001A1B1C1DAFB1B0B5000904020001030068
:100250000000092101010001226500070584034017
:10026000000105010902A1010901A100850105099B
:1002700019012903150025019503750181029501D6
:100280007505810305010930093109381581257F7C
:10029000750895038106C0C005010906A101850204
:1002A000050719E029E71500250175019508810268
:1002B00095017508810395067508150025650507E4
:1002C000190029658100C000B7070A0911241FBE63
:1002D000CFEFDAE0DEBFCDBF11E0A0E0B1E0EEE8A5
:1002E000F2E102C005900D92A832B107D9F721E0E2
:1002F000A8E2B1E001C01D92A739B207E1F712E010
:10030000CCECD2E004C02297FE010E944109C83C17
:10031000D107C9F70E9440030C9445090C940000D2
:1003200061E08DE00C94D00261E08DE00E94090351
:1003300068EE73E080E090E00E94150260E08DE0DE
:100340000E94090368EE73E080E090E00C941502CF
:100350001F920F920FB60F9211242F933F938F93FA
:100360009F93AF93BF938091290190912A01A0910F
:100370002B01B0912C013091280123E0230F2D3760
:1003800020F40196A11DB11D05C026E8230F029699
:10039000A11DB11D209328018093290190932A016A
:1003A000A0932B01B0932C0180912D0190912E01EF
:1003B000A0912F01B09130010196A11DB11D809334
:1003C0002D0190932E01A0932F01B0933001BF9186
:1003D000AF919F918F913F912F910F900FBE0F90F2
:1003E0001F9018953FB7F89480912D0190912E01A0
:1003F000A0912F01B091300126B5A89B05C02F3FD9
:1004000019F00196A11DB11D3FBF6627782F892FD6
:100410009A2F620F711D811D911D42E0660F771F9B
:10042000881F991F4A95D1F70895CF92DF92EF92D6
:10043000FF92CF93DF936B017C010E94F201EB01ED
:10044000C114D104E104F10489F00E94F9060E946C
:10045000F2016C1B7D0B683E734090F381E0C81A7B
:10046000D108E108F108C851DC4FEACFDF91CF9104
:10047000FF90EF90DF90CF900895789484B58260DC
:1004800084BD84B5816084BD85B5826085BD85B538
:10049000816085BDEEE6F0E0808181608083E1E8E7
:1004A000F0E010828081826080838081816080831F
:1004B000E0E8F0E0808181608083E1E9F0E0808124
:1004C00082608083808181608083E0E9F0E08081C8
:1004D00081608083E1ECF0E08081846080838081B2
:1004E00082608083808181608083E3ECF0E08081A2
:1004F00081608083E0ECF0E0808182608083E2ECC8
:10050000F0E0808181608083EAE7F0E080818460B0
:10051000808380818260808380818160808380810C
:1005200080688083089590E0FC013197EF30F105F9
:10053000B0F5EA5AFF4F0C943F09809180008F7705
:1005400003C0809180008F7D80938000089580910A
:100550008000877FF9CF84B58F7702C084B58F7D07
:1005600084BD0895809190008F7707C0809190009E
:100570008F7D03C080919000877F809390000895C5
:100580008091C0008F7703C08091C0008F7D8093E1
:10059000C00008958091C200877F8093C2000895B3
:1005A000CF93DF9390E0FC01E851FF4F2491FC01D1
:1005B000EA5FFE4F8491882349F190E0880F991FEC
:1005C000FC01EE5CFE4FA591B4918C5D9E4FFC0149
:1005D000C591D4919FB7611108C0F8948C91209572
:1005E00082238C93888182230AC0623051F4F8946C
:1005F0008C91322F309583238C938881822B888332
:1006000004C0F8948C91822B8C939FBFDF91CF9183
:1006100008950F931F93CF93DF931F92CDB7DEB74B
:10062000282F30E0F901E653FF4F8491F901E8519A
:10063000FF4F1491F901EA5FFE4F04910023C9F0C6
:10064000882321F069830E9493026981E02FF0E002
:10065000EE0FFF1FEC5DFE4FA591B4919FB7F8948C
:100660008C91611103C01095812301C0812B8C9363
:100670009FBF0F90DF91CF911F910F910895089523
:100680000E943D020E943F0381E391E00E94D9064F
:100690000E949001C0E0D0E00E9494012097E1F315
:1006A0000E940000F9CF4091350150913601209110
:1006B00033013091340142175307B4F49091E800AC
:1006C0009570E1F39091E80092FD19C08093F100DC
:1006D000809135019091360101968F739927892B6E
:1006E00019F48EEF8093E8008091350190913601E6
:1006F0000196909336018093350181E0089580E062
:100700000895CF92DF92FF920F931F93CF93DF93C1
:100710001F92CDB7DEB7082F162F862F880F8E5F5A
:1007200099830E94530383E00E945303F02EC02E4E
:100730009981D92E8C2D8F19811778F4F601849127
:100740000E945303082F80E00E9453038023FFEF91
:10075000CF1ADF0A8111EECF01C081E00F90DF9147
:10076000CF911F910F91FF90DF90CF90089561502E
:1007700030F02091F100FC0120830196F8CF289AF7
:1007800084E68093380108952FB7FC012083F89404
:1007900067706093E9000895CF93DF931F92CDB700
:1007A000DEB7682FCE0101960E94C4038091F2004B
:1007B00099819FBF0F90DF91CF910895FF920F9382
:1007C0001F93CF93DF9300D0CDB7DEB7F62E8A010B
:1007D00090913701992311F057FF03C08FEF9FEFDE
:1007E0002BC0682FCE0101967A830E94C4038091AA
:1007F000F20090E0A8017A81801791070CF4AC0117
:10080000EF2DF72FF40E84E6FE1639F0289A809328
:1008100038019091F1009193F7CF4115510521F0E6
:100820008091F200882321F089818FBFCA0104C022
:100830008BE68093E800F8CF0F900F90DF91CF9177
:100840001F910F91FF900895CF93DF931F92CDB723
:10085000DEB741E050E0BE016F5F7F4F0E94DE03D4
:10086000019719F4898190E002C08FEF9FEF0F90FC
:10087000DF91CF910895CF93DF931F92CDB7DEB76D
:10088000682FCE0101960E94C4039091E800892F41
:10089000807295FF04C09091F20080E4891B9981D9
:1008A0009FBF0F90DF91CF9108956F927F928F92AB
:1008B0009F92AF92BF92CF92DF92EF92FF920F93EF
:1008C0001F93CF93DF931F92CDB7DEB7782E7B01B6
:1008D000C42EB52E80913701882369F0042F152F7F
:1008E0008AEFD82E872D8072982E9AE3A92E872D15
:1008F0008074882E11C08FEF9FEF57C0872D0E9404
:100900003B04682E81110CC0DA94A9F361E070E019
:1009100080E090E00E9415020115110579F73BC0B7
:10092000282F30E0021713070CF4602E672DCE013C
:1009300001960E94C4038091E80085FF29C0262DFE
:1009400030E0021B130B992039F06A948FEF681680
:10095000B1F01092F100F9CFF701862D77FE07C0B4
:10096000815058F094919093F1003196F9CF8150D5
:1009700020F091919093F100FACFE20EF31E809156
:10098000E80085FF0FC00115110511F481100AC0A0
:1009900089818FBFC1CF5D9A84E6809339018C2D08
:1009A0009B2D03C0A092E800F3CF0F90DF91CF9171
:1009B0001F910F91FF90EF90DF90CF90BF90AF907D
:1009C0009F908F907F906F9008951092E900109201
:1009D00036011092350190933401809333010895CC
:1009E000CF92DF92FF920F931F93CF93DF9300D0AC
:1009F000CDB7DEB7F82E8A016B0101151105B1F0F4
:100A0000F601F7FE02C0849101C0808149835A83B8
:100A10000E94530301501109FFEFCF1ADF0A4981E9
:100A20005A818111EACF8FEF9FEF01C0CA010F9069
:100A30000F90DF91CF911F910F91FF90DF90CF909A
:100A400008951F93CF93DF931F92CDB7DEB7162F74
:100A50002091E80022FFFCCF612F79830E94B70329
:100A60008BEF8093E800812F7981972F0F90DF9192
:100A7000CF911F910895CF93DF931F92CDB7DEB72B
:100A80001982CE0101960E945707CE0101960E945D
:100A9000F207898190E00F90DF91CF9108951F9226
:100AA0000F920FB60F921124EF92FF920F931F93A4
:100AB0002F933F934F935F936F937F938F939F9366
:100AC000AF93BF93EF93FF93CF93DF93CDB7DEB791
:100AD0006297DEBFCDBF1092E9008091E80083FFEE
:100AE000EBC068E0CE010A960E94B70382EF8093C4
:100AF000E8009A8597FF05C08091E80080FFFCCF51
:100B000003C08EEF8093E800892F807609F0B9C08A
:100B10008B85811105C01092F1001092F100C5C0C3
:100B2000282F2D7F213009F4C0C0853049F48091F1
:100B3000E80080FFFCCF8C8580688093E300B5C01F
:100B4000863009F076C02D85E888F988223071F565
:100B500080E090E02A8B0E94E5040E943B0599E02A
:100B60008E010F5F1F4FF801392F11923A95E9F767
:100B700099832A892A8391E09E8390E898879AEF47
:100B800099872091350130913601275F3F4F3C8393
:100B90002B838D83C7010E94E50449E050E0B80132
:100BA00080E00E94F0040E943B057FC0C7012A8BB1
:100BB0000E94E5042A89223241F482E290E00E94F8
:100BC000FD07892B09F071C074C0213069F4888950
:100BD0009989089711F42093320180913201811193
:100BE00018C067E571E01AC0233009F062C08C8537
:100BF000882391F0823021F46DE085E791E006C012
:100C0000813009F056C06BE089E691E00E948103D3
:100C10004AC065E471E002C063E871E061157105E6
:100C200009F447C0FB01449150E080E80E94F004C1
:100C30003CC0873009F43DC0883021F481E08093C6
:100C4000F10033C0893089F5937099F5E1E4F1E062
:100C500081E021E096E38093E9002093EB0034915A
:100C60003093EC009093ED008F5F3196853099F7CB
:100C70008EE78093EA001092EA008C85809337011A
:100C800014C0888999890E94E5048E85811105C068
:100C9000CE010A960E94620706C0823051F4CE014E
:100CA0000A960E942508882321F08EEF8093E800A1
:100CB00003C081E28093EB0062960FB6F894DEBF2A
:100CC0000FBECDBFDF91CF91FF91EF91BF91AF915B
:100CD0009F918F917F916F915F914F913F912F9154
:100CE0001F910F91FF90EF900F900FBE0F901F90EC
:100CF00018958093E9008091F200882319F08AE327
:100D00008093E80008951F920F920FB60F9211245E
:100D10002F933F934F935F936F937F938F939F9303
:100D2000AF93BF93EF93FF938091E1001092E100A6
:100D300083FF0FC01092E90091E09093EB001092B6
:100D4000EC0092E39093ED001092370198E09093BD
:100D5000F00082FF1DC083E00E9479068091390176
:100D6000882339F08091390181508093390188239B
:100D700069F080913801882359F0809138018150C1
:100D800080933801811104C0289802C05D98F1CF8A
:100D9000FF91EF91BF91AF919F918F917F916F9153
:100DA0005F914F913F912F910F900FBE0F901F9029
:100DB00018951092370181E08093D70080EA8093E4
:100DC000D80082E189BD09B400FEFDCF61E070E08A
:100DD00080E090E00E94150280E98093D8008CE0CA
:100DE0008093E2001092E000559A209A5D9828982E
:100DF00008950895CF93DF931F92CDB7DEB769832F
:100E0000DC01ED91FC910280F381E02D41E050E0A6
:100E1000BE016F5F7F4F09950F90DF91CF910895CD
:100E2000CF93DF93EC018C859D8597FF05C082E011
:100E30000E9424049D878C878C859D85DF91CF91AE
:100E4000089583E00C947906FC018485958597FDCF
:100E500006C082E00E94CC0390E00196089582E0F3
:100E60000E94CC0390E00895FC018485958597FD50
:100E700005C02FEF3FEF35872487089582E00C945B
:100E80002404CF93DF93EC0180910701882331F094
:100E900083E00E9455041816190634F081E090E0B2
:100EA0009B838A8380E090E0DF91CF910895FC01DD
:100EB00020812E5F208342E450E067E871E080E803
:100EC0000C94F004FC0181819081913A59F48132B3
:100ED00009F03CC047E050E060E071E080E00E9433
:100EE000F00443C0913291F5803239F467E070E04C
:100EF00080E091E00E94210506C0823209F035C0F1
:100F00008281809307018091000190910101A0915D
:100F10000201B0910301803B9440A105B105C1F4E9
:100F20008091070180FD14C087E797E7909301083F
:100F3000809300082BE088E190E00FB6F894A89524
:100F4000809360000FBE209360000FC080E0089582
:100F500088E10FB6F89480936000109260000FBE95
:100F6000A895109201081092000881E0089510924F
:100F70003D0110923C0188EE93E0A0E0B0E0809348
:100F80003E0190933F01A0934001B09341018EE058
:100F900091E090933B0180933A018FEF9FEF909304
:100FA0004701809346010895FF920F931F93CF93BB
:100FB000DF93EC01F62EE881F9810480F581E02DC4
:100FC00009958C01E881F9810680F781E02D6F2D6C
:100FD000CE010995C8019927DF91CF911F910F91FB
:100FE000FF900895FC0120812F5F208349E150E0AC
:100FF00069E472E080E80C94F00445E650E062E6B3
:1010000072E080E80C94F004EF92FF920F931F932C
:10101000CF93DF931F92CDB7DEB789838B017A011F
:1010200041E050E0BE016F5F7F4F84E00E945504B5
:10103000A701B80184E40E9455040F90DF91CF917D
:101040001F910F91FF90EF900895FC019181808195
:10105000813A31F481E0913091F0933089F411C0FC
:10106000813271F49B3021F482818093090105C0A3
:101070009A3031F482818093080181E008950895C7
:1010800080E0089548E050E082E00C940408CF939B
:10109000DF93DC01683818F0E8E7E60F25C0E62F9B
:1010A000F0E067FF11C0E058F10981E090E001C075
:1010B000880FEA95EAF714969C911497982B14964A
:1010C0009C931497E0E010C0E753FE4FE491EE23A9
:1010D00009F440C0E7FF08C014968C911497826011
:1010E00014968C931497EF7716968C9116978E170B
:1010F00041F117968C9117978E1719F118968C91CC
:1011000018978E17F1F019968C9119978E17C9F0D0
:101110001A968C911A978E17A1F01B968C911B979B
:101120008E1779F080E090E0ED01C80FD91F2E8175
:10113000211102C0EE8305C0019686309105A1F70A
:1011400009C0BD016C5F7F4FCD010E94420881E064
:1011500090E008C081E090E013969C938E931297E4
:1011600080E090E0DF91CF910895683818F0E8E7CB
:10117000E60F25C0E62FF0E067FF12C0E058F10946
:1011800021E030E001C0220FEA95EAF72095DC016A
:1011900014963C911497322314963C93E0E00FC0D0
:1011A000E753FE4FE491EE2329F1E7FF08C0DC018D
:1011B00014962C9114972D7F14962C93EF7720E0A2
:1011C00030E0EE2351F0DC01A20FB31F16964C91D4
:1011D00016974E1302C016961C922F5F3F4F263073
:1011E000310579F7BC016C5F7F4F0E94420881E0B6
:1011F00090E0089580E090E00895FC011682178247
:1012000010861186128613861482BC016C5F7F4F94
:101210000C9442081092960110928D0110928C014C
:101220008EE191E090938B0180938A010895CF9293
:10123000DF92EF92FF920F931F93CF93DF936C0196
:101240007A01EB01E60EF71E00E010E0CE15DF0597
:1012500061F06991D601ED91FC910190F081E02D52
:10126000C6010995080F191FF1CFC801DF91CF9171
:101270001F910F91FF90EF90DF90CF900895EE0FA8
:0E128000FF1F0590F491E02D0994F894FFCF24
:10128E0000E1000000000000010100000000FA066D
:10129E004107240734071007210700000000D40778
:0812AE0017094708B508FD0807
:00000001FF
